:100000000C94F4030C942C040C942C040C942C04E9
:100010000C942C040C942C040C942C040C942C04A0
:100020000C942C040C942C040C9414290C94E829A2
:100030000C9454230C942C040C942C040C942C0439
:100040000C942C040C942C040C942C040C942C0470
:100050000C942C040C94DB230C942C040C942C0492
:100060000C942C040C942C040C942C040C942C0450
:100070000C942C040C942C040C942C040C942C0440
:100080000C942C040C942C040C942C040C942C0430
:100090000C942C040C942C040C942C040C942C0420
:1000A0000C942C040C942C040C942C0429003A007D
:1000B0003B003C003D003E003F004000410042004C
:1000C000430044004500460049004C0035001E0036
:1000D0001F0020002100220023002400250026000C
:1000E00027002D002E0000002A004A002B000000EF
:1000F00014001A000800150017001C0018000C005E
:10010000120013002F00300031004B0039000000B6
:1001100004001600070009000A000B000D000E0085
:100120000F0033003400000028004E00E100000002
:100130001D001B000600190005001100100036000C
:10014000370038000000E50052004D00E000E300F9
:10015000E2000000000000002C0000000000000091
:1001600001510000E400500051004F00005C01000C
:100170000100010001000100010001000100010077
:100180000100010001000100010001000100010067
:100190000100010001000100010001000100010057
:1001A0000100010001000000010001000100000049
:1001B0000100010001000100010001000100010037
:1001C0000100010001000100010001000100000028
:1001D0000100010001000100010001000100010017
:1001E0000100010001000000010001000100000009
:1001F000C25CC35CC55CC65CC75CC85CC95CCA5CED
:1002000001000100000001000100010001000100E7
:1002100001000000000000000100000000000000DC
:10022000010000000100010001000100005C01006C
:1002300001000100010001000100010001000100B6
:1002400001000100010001000100010001000100A6
:100250000100010001000100010001000100010096
:100260000100010001000000010001000100000088
:100270000100010001000100010001000100010076
:100280000100010001000100010001000100000067
:100290000100010001000100010001000100010056
:1002A0000100010001000000010001000100000048
:1002B0000100010001000100010001000100010036
:1002C0000100010000000100010001000100010027
:1002D000010000000000000001000000000000001C
:1002E000010000000100010001000100005C0100AC
:1002F00001000100010001000100010001000100F6
:1003000001000100010001000100010001000100E5
:1003100001000100010001000100010001000100D5
:1003200001000100010000000100010001000000C7
:1003300001000100010001000100010001000100B5
:1003400001000100010001000100010001000000A6
:100350000100010001000100010001000100010095
:100360000100010001000000010001000100000087
:100370000100010001000100010001000100010075
:100380000100010000000100010001000100010066
:10039000010000000000000001000000000000005B
:1003A0000100000001000100010001000000000048
:1003B000000000002A2B28000000000000000000C0
:1003C0000000000000000029000000002C1E342066
:1003D000212224342627252E362D3738271E1F208C
:1003E0002122232425263333362E37381F040506D1
:1003F0000708090A0B0C0D0E0F1011121314151615
:100400001718191A1B1C1D2F3130232D3504050612
:100410000708090A0B0C0D0E0F10111213141516F4
:100420001718191A1B1C1D2F3130354C0000000005
:1004300000000000000000000000000000000000BC
:1004400000000000000000000000000000000000AC
:100450007E0F00D4FFFFFFC7000000781E0F0500CD
:10046000047F3F1F643214643214783C1E1E140A49
:10047000052223252628292A2C2D2F3032333536E4
:10048000383A3B3D3E4042434547494A4C4E505125
:10049000535557595A5C5E6062646668696B6D6F4C
:1004A00071737577797B7D7F81838587898A8C8E4F
:1004B00090929496989A9C9E9FA1A3A5A7A8AAAC57
:1004C000AEAFB1B3B4B6B8B9BBBCBEBFC1C2C3C591
:1004D000C6C7C9CACBCCCDCED0D1D2D2D3D4D5D633
:1004E000D7D7D8D9D9DADADBDBDBDCDCDCDCDCDD66
:1004F000DDDDDDDCDCDCDCDCDBDBDBDADAD9D9D84A
:10050000D7D7D6D5D4D3D2D2D1D0CECDCCCBCAC9E1
:10051000C7C6C5C3C2C1BFBEBCBBB9B8B6B4B3B110
:10052000AFAEACAAA8A7A5A3A19F9E9C9A989694AB
:1005300092908E8C8A89878583817F7D7B79777580
:1005400073716F6D6B6968666462605E5C5A59575F
:10055000555351504E4C4A4947454342403E3D3B1E
:100560003A3836353332302F2D2C2A2928262523A8
:1005700022FFAA7F55400001010101010101010193
:100580000202020202020202020303030303030344
:100590000304040404040404050505050506060611
:1005A0000606070707070708080808090909090ACE
:1005B0000A0A0B0B0B0C0C0C0D0D0D0E0E0E0F0F73
:1005C0000F10101111111212131314141515161601
:1005D0001717181819191A1A1B1B1C1D1D1E1E1F70
:1005E0002020212222232424252626272829292ABF
:1005F0002B2C2D2D2E2F30313232333435363738E7
:10060000393A3B3C3D3E3F404142434445464748E2
:10061000494A4C4D4E4F50515354555658595A5BB8
:100620005D5E5F616264656668696B6C6D6F707258
:10063000737577787A7B7D7E8082838587888A8CC4
:100640008E8F91939596989A9C9EA0A2A3A5A7A9F8
:10065000ABADAFB1B3B5B7BABCBEC0C2C4C6C9CBEF
:10066000CDCFD1D4D6D8DBDDDFE2E4E7E9EBEEF0A5
:10067000F3F5F8FAFDFF120342006F0075007200F7
:10068000670065006100750000001C0353007400E2
:100690007500640069006F0020004B006500730066
:1006A00074007200610000000403090409025B0089
:1006B000030100A0FA09040000010301010009215F
:1006C000110100012240000705810308000109040F
:1006D0000100020300000009211101000122220093
:1006E0000705820320000107050303200001090418
:1006F00002000103000000092111010001226D0028
:100700000705840320000112010002000000081008
:100710007C01750100010200010660FF0961A10171
:100720000962150026FF00952075088102096315EE
:100730000026FF00952075089102C005010980A1DF
:1007400001850319012AB700150126B70095017527
:10075000108100C0050C0901A101850419012AA01E
:1007600002150126A002950175108100C00501093E
:1007700006A1018506050719E029E7150025019561
:1007800008750181020507190029EF15002501955B
:10079000F07501810205081901290595057501917A
:1007A00002950175039101C005010906A101050724
:1007B00019E029E7150025019508750181029501C9
:1007C000750881010507190029FF150026FF00950E
:1007D000067508810005081901290595057501911F
:1007E00002950175039101C011241FBECFEFDAE01D
:1007F000DEBFCDBF04B603FE18C08091C603909142
:10080000C703A091C803B091C9038730904BA7409C
:10081000B04B59F41092C6031092C7031092C8034C
:100820001092C903E0E0F8E3099511E0A0E0B1E01F
:10083000EEE5FBE502C005900D92A83DB107D9F7A2
:1008400023E0A8EDB1E001C01D92A63CB207E1F79C
:100850000E94A1130C94452D0C94000081E0089592
:1008600081E008950E943004089508950E9435049F
:100870000895A5E0B0E0EFE3F4E00C94402C498348
:100880005A833091DB0189819A81311119C0662325
:1008900099F0222389F00E94C50A182F682F8981B8
:1008A0009A810E94A20A69817A81812F0E945A202E
:1008B0002596E3E00C945C2C0E94B30A182FF3CF2A
:1008C0000E94C50A69817A81F1CFFC01262F4081FF
:1008D00051816281738184810E943904089581E08D
:1008E0000895CF93DF93EC0160E00E946504BE01A0
:1008F0000E943604DF91CF910895E1E0F0E0DF013E
:1009000002C0AA0FBB1F6A95E2F7BD01DF0102C05A
:10091000AA0FBB1F4A95E2F76A2B01C0EE0F2A957A
:10092000EAF7962F9823961302C08E2B0895E09530
:100930008E230895242F462F682F809100020E9455
:100940007D040E94020A08950E944C1208950E949C
:100950005012089508950E949F090E94AA042FEF43
:1009600084E39CE0215080409040E1F700C000000B
:1009700008950E94AB040E94FF2308950E94AB04D7
:100980000E94232408950F931F93CF93DF938C012C
:1009900061E00E946504EC01B8010E945B1C8111BA
:1009A00006C080E0DF91CF911F910F910895B801AB
:1009B000CE010E9432048823A1F3B801CE010E9427
:1009C0009D21882371F3B801CE010E94A71D8823C1
:1009D00041F3B801CE010E940F21882311F3B80121
:1009E000CE010E94001B8823E1F2F8018281882356
:1009F00061F0CA35FDE5DF0701F158F4C115ECE5FA
:100A0000DE0791F0CE3DDC4591F0C8010E942E0436
:100A1000C9CFCC358DE5D80769F090F0C73ADD45F0
:100A2000A1F70E94BE04BDCF0E94B904BACF0E94B4
:100A30007E0FF7CF0E94B80EE8CF0E94C20EE5CF1E
:100A40000E94C60EE2CF0E9430230E940B060E9435
:100A5000661908950E940F060E943D1A0E943523D0
:100A60000895B0E0A0E0E7E3F5E00C943C2CE82F1B
:100A7000F0E0E455FC4FD490282F26952695269536
:100A800030E0F901E45BFB4F0491877010E0082E21
:100A900002C0159507950A94E2F701701127F90134
:100AA000E45CFB4FE490F12C082E02C0F594E7942F
:100AB0000A94E2F791E0E922FF24F901E45DFB4F9B
:100AC000C491D0E002C0D595C7958A95E2F7C17070
:100AD000DD270115110519F081EE0E945A06E11477
:100AE000F10419F086EE0E945A068D2D0E945107DE
:100AF000E114F10419F086EE0E94E80601151105D3
:100B000019F081EE0E94E806CD2B19F08CE20E94CC
:100B10005107CDB7DEB7E7E00C94582CEF92FF9267
:100B20000F931F93CF93DF93EC01162F0AE0888178
:100B3000882309F454C0813009F04EC08981813086
:100B400099F47E0122E0E20EF11C8A810E94510795
:100B5000E7012196812F815050F3EFE9FFE03197B3
:100B6000F1F700C00000F7CF823041F47E0182E04F
:100B7000E80EF11C8A810E945A06EACF833041F4C4
:100B80007E01E2E0EE0EF11C8A810E94E806E0CFD1
:100B9000843011F02196DDCF2A81229690E080E00A
:100BA000AE014F5F5F4F2053330B2A30310548F0C1
:100BB000019778F2EFE9FFE03197F1F700C000000C
:100BC000F7CF089FB001099F700D1124C901860F4E
:100BD000971F2981EA01E4CF0E943105BACFCDB732
:100BE000DEB7E6E00C94592C60E00E948E05089573
:100BF00008950E94F805089581E008950E94FC057B
:100C000008950895CF93C82F0E94F9058C2F0E9454
:100C1000FE05CF91089580E00E94020608950E948B
:100C2000F9210E94020608950E94F9219091DA01AB
:100C3000981721F08093DA010E9402060895ABE034
:100C4000B0E0E5E2F6E00C94412C4F8358876987C9
:100C50007A878B8761110E94030E1E821D8285E0B8
:100C6000FE013796DE01119601900D928A95E1F70B
:100C70008C819D81892B61F449815A816B817C81B2
:100C80008D819E810E942C0D2B96E2E00C945D2CB0
:100C900089819A8189238F3F79F3CE0101960E9441
:100CA0006F048111E9CFF0CFFC01808191810E9416
:100CB000F20A0895CF93C82F8823C9F08238C9F467
:100CC0000E94F92181FD13C089E30E94BB0D0E949F
:100CD000240E2FEF81EE94E0215080409040E1F708
:100CE00000C0000089E30E94C30D0E94240ECF9132
:100CF00008958338A1F40E94F92180FDF8CF83E59F
:100D00000E94BB0D0E94240E2FEF81EE94E0215033
:100D100080409040E1F700C0000083E5E4CF8438D4
:100D2000A1F40E94F92182FDE2CF87E40E94BB0D6D
:100D30000E94240E2FEF81EE94E0215080409040DD
:100D4000E1F700C0000087E4CECF8CEF8C0F813A32
:100D5000B8F48C2F0E94521F8111C9CF6C2F809143
:100D60000401909105010E946022882329F08C2FB4
:100D70000E94C30D0E94240E8C2F0E94BB0DB5CF84
:100D800080E28C0F883048F4C77081E001C0880F82
:100D9000CA95EAF70E94E60DA8CFEBE5EC0FE33029
:100DA00040F4F0E0EC5AFE4F808190E00E94202257
:100DB0009ECFC85AC73108F09ACFEC2FF0E0EE0F63
:100DC000FF1FEA5DFE4F808191810E9436228FCF06
:100DD000882309F44DC0823879F40E94F92181FFFB
:100DE00047C089E30E94BB0D0E94240E89E30E9444
:100DF000C30D0E94240E0895833859F40E94F921EE
:100E000080FF36C083E50E94BB0D0E94240E83E55F
:100E1000EECF843859F40E94F92182FF29C087E47B
:100E20000E94BB0D0E94240E87E4E1CF9CEF980F37
:100E3000913AE8F290E2980F983050F4877091E080
:100E400001C0990F8A95EAF7892F0E94EC0DD1CF46
:100E50009BE5980F933028F490E080E00E942022D8
:100E60000895885A873120F490E080E00E9436226D
:100E700008951F93CF93DF93182FEB010E945A061A
:100E8000209739F4812F0E94E806DF91CF911F91BE
:100E900008958FE99FE00197F1F700C000002197C6
:100EA000EFCF70E060E0893311F460E570E00E94FC
:100EB00039070895882321F00E94E60D0E94240E30
:100EC0000895882321F00E94EC0D0E94240E0895BD
:100ED000B0E0A0E0EEE6F7E00C943A2C6C01D62FDF
:100EE000C72FFC011281F580F2949FE0F9220E9445
:100EF000DC0DE82E8823B9F0E12E1123A1F08C2F10
:100F0000807F803421F080E28D0F8830D0F0809196
:100F10004F0382FF16C082E00E94870E0E94DC0D04
:100F200091E0E82EE926BC2EB2948FE0B822FBE0D7
:100F3000FB1508F468C0EB2DF0E0E95BF24D0C9472
:100F4000F32BE12CF0CF0C2F0F70C07F11F0029526
:100F5000007F112399F0002359F080E28D0F883033
:100F600010F0D11107C0802F0E94E60D0E94240EC0
:100F70008D2F41C0802F0E94F60DF8CF8D2F0E943B
:100F8000E806002309F43FC080E28D0F883010F09E
:100F9000D11104C0802F0E94EC0D03C0802F0E944D
:100FA000FC0D0E94240E2FC00C2F0F70C07FC0328A
:100FB00011F00295007FDD2381F0D13009F463C088
:100FC000112309F46DC0FF2009F463C0F601858187
:100FD00080FFCECF8F7085835CC080914F0382FDF0
:100FE00033C0112359F0002329F0802F0E94E60D11
:100FF0000E94240E80E00E945A0605C080E00E94F4
:10100000E8060111C7CFEB2DE850FF0B349720F411
:101010000E94F9210E940206EE2089F00E94D80D5C
:1010200080FD0DC0F60112820E94D20D0E94160AA8
:10103000C6010E9463090E94D20D0E94220ACDB708
:10104000DEB7E9E00C94562C112389F0F11006C0AC
:101050000E94060E802B0E945A07D5CF21E0F21283
:10106000F7CF0E94060E802B0E940D0ECCCFF11000
:1010700006C00E941A0E802F0E946107C4CF31E083
:10108000F31609F2F6CF112331F085E08F1508F43D
:10109000BACF802FE0CF94E09F1508F4B4CFEBCF08
:1010A000FF2049F3D93349F4FFEF27EE33E0F15045
:1010B00020403040E1F700C000008D2F0E94E8067C
:1010C000A2CF8C2F86958695837069F0813009F0C8
:1010D0009ACF8D2F9C2F9370111102C090E080E069
:1010E0000E94362290CF8D2F9C2F9370111102C039
:1010F00090E080E00E94202286CF8C2F837079F5CB
:10110000111181CF4D2F429546954770440F440FE2
:101110008D2F8F70042E01C0880F0A94EAF72D2FAF
:101120002071D4FF07C02FE030E001C0220F4A95A4
:10113000EAF72095C695C695C370822BC23049F058
:1011400058F4C13019F00E94F0095DCF0E94EA09FD
:101150005ACF0E94F60957CF0E94E70954CF8695CF
:10116000112311F08C2F8170882309F44CCF4D2F5F
:10117000429546954770440F440F8D2F8F70042E73
:1011800001C0880F0A94EAF72D2F2071D4FF07C001
:101190002FE030E001C0220F4A95EAF72095C6956E
:1011A000C695C370822BC23049F058F4C13019F093
:1011B0000E94410A28CF0E943B0A25CF0E94470A7D
:1011C00022CF0E94020A1FCFCF70112329F08C2F4B
:1011D0000E94160A8D2F3FCF8D2F0E9461078C2F02
:1011E0000E94220A10CFD23F51F160F4D03FB9F0F3
:1011F000D13F81F0112309F449C0F110B9CE8C2FF1
:101200008F7121C0D33F11F1D43FA1F780914F03DB
:1012100082FD26C08C2F8F71112311F314C011236E
:1012200049F084E08F1508F4EECE8C2F8F710E9468
:101230002F0AE9CE95E09F1508F4E5CEF6CF8C2F66
:101240008F711111CDCF0E94160ADDCE112329F026
:101250008C2F8F710E940D0AD6CE0E94090AD3CE20
:10126000112349F0CF718C2F0E94160A63E08C2F56
:101270000E94690EC8CE81E00E94870EE1E0EF1562
:1012800008F0C1CE82E00E94870EBDCEF1100ACFD9
:101290008C2F8F71A5CF0F931F93CF93DF93EC010A
:1012A000688179818A810E94FD0A8C010E944D0A21
:1012B0000E94E609B801CE010E946807DF91CF9134
:1012C0001F910F910895CF93DF93EC018B819C8147
:1012D000892B29F08881998189238F3F51F4DF91EF
:1012E000CF910895CE010E944B09CE010E94710456
:1012F000F6CFCE010E94C3048111F4CF0E94DC0D11
:10130000882369F38A81882351F380914F0382FFF8
:10131000E6CF82E00E94870EE2CF90E080E00E945C
:10132000202290E080E00E9436220E94030E0E945C
:10133000240E08950E94CB0D0E948D0908950E94ED
:10134000F30D0E949A09089592959F70963091F03E
:1013500058F4925F9F70923058F4803F19F030F447
:10136000883E30F481E008959A5FF4CF843FD1F352
:1013700080E00895883EB0F3813FD1F7F3CFFC01C0
:10138000808191810E94F20A0E94A4090895A5E03B
:10139000B0E0EDECF9E00C94412C2596E2E00C94E1
:1013A0005D2CA6E0B0E0E7EDF9E00C94412C269628
:1013B000E2E00C945D2C08950E94DB0908950E94E0
:1013C000DC09809301020E948D09089508950E940E
:1013D000DF09089590910102892B0E94DF09089589
:1013E0009091010289230E94DF09089590910102E2
:1013F00089270E94DF0908950E94DB0908950E9451
:10140000FC0908950E94FF09809300020E948D0943
:10141000089580E00E94020A089591E001C0990FAA
:101420008A95EAF7892F0E94020A089521E030E0A8
:1014300001C0220F8A95EAF780910002822B0E9458
:10144000020A089521E030E001C0220F8A95EAF7F0
:1014500020958091000282230E94020A089521E0D3
:1014600030E001C0220F8A95EAF7809100028227BE
:101470000E94020A089590910002892B0E94020A9C
:1014800008959091000289230E94020A0895909184
:10149000000289270E94020A08950895262F2770C6
:1014A00091E001C0990F2A95EAF723E076956795B8
:1014B0002A95E1F7FB01EE0FFF1FE60FF71FE40F80
:1014C000F51F50E040E0682F70E08191DF01119737
:1014D0009B01042E02C0369527950A94E2F72170ED
:1014E00021952827292328272C934F5F5F4F4330CE
:1014F000510559F70895A82FA77023E09695879571
:101500002A95E1F7FC01EE0FFF1FE80FF91FE60F28
:10151000F71F50E040E080E0219130E00A2E02C049
:10152000369527950A94E2F721703327042E01C0DF
:10153000220F0A94EAF7822B4F5F5F4F4330510529
:1015400059F70895262F963068F4803158F430E129
:10155000939FB0011124680F711D4CED51E0822F53
:101560000E944E0A0895963070F4803160F440E194
:10157000949F900111246CED71E0820F932F911DC7
:101580000E947B0A089580E00895CF92DF92FF9237
:101590000F931F93CF93DF936C0100910002809112
:1015A0000102082BC7E0D0E010E0FC2EC8010C2E91
:1015B00002C0959587950A94E2F780FD0CC02197AB
:1015C000A0F7F12C8F2DDF91CF911F910F91FF90FC
:1015D000DF90CF900895B6018C2F0E9435110197AE
:1015E00071F3F0CFCF93DF93EC010E94C50ABE01E7
:1015F0000E943511DF91CF9108951F93CF93DF9310
:10160000EB019091DB01992339F0CB010E94F20AA2
:10161000DF91CF911F910895882369F0CB010E943B
:10162000C50A182F682FCE010E94A20ABE01812F81
:101630000E943511EDCFCB010E94B30A182FF6CFCF
:101640001F93CF93DF93C091020216E080910302B3
:101650008C1304C0DF91CF911F910895D0E01C9F9F
:10166000F0011D9FF00D1124EC5FFD4F4081518171
:1016700062817381848195810E94D1092196C7700E
:10168000E5CF40913402509135026091360270915D
:10169000370280913802909139020E94D109089551
:1016A0001F93CF93DF9380913902807F09F049C067
:1016B00080913602882309F444C080910202C091CF
:1016C00003026091340270913502A0913702B0910B
:1016D0003802D62FD72316E0C81799F190E010975B
:1016E00011F0DF3F19F401968770F6CF189F900133
:1016F000199F300D1124F901EC5FFD4F4181471313
:10170000F2CF40814613EFCF42814111ECCF4381AC
:1017100054814A1B5B0B483C510528F780913902E4
:101720008F70806180933902F901E75FFD4F8081FE
:101730008F708061808384E392E00E9463090E943D
:10174000200BDF91CF911F910895A1E1B0E0EBEA6A
:10175000FBE00C94392C8C0185E0F801DE011D962C
:1017600001900D928A95E1F7F801E28084E3C82E9A
:1017700082E0D82E609137027091380261157105B0
:1017800009F44EC19091340220913502892F8223B1
:101790008F3F09F445C140815181A380B480F0900E
:1017A0003602F501E61BF70BFF2009F4EAC0809131
:1017B0003902382F307FE83CF10508F0A3C0311121
:1017C0006DC0FE2C251316C0941314C0E11012C076
:1017D0008F708061809339020E94410BC6010E9484
:1017E000630980913902F80185838F2D6196EAE0C3
:1017F0000C94552CA114B10429F0842F85238F3F1C
:1018000009F027C180E0F82FF170DF2E80FF3CC087
:10181000809102022091030236E0821315C04D87A9
:101820005E878D859E850E94F20A292F22952F7052
:101830002230F0F0243018F59F70F1F0F801958116
:10184000907FD1F4D12C1EC090E0389FF001399FD9
:10185000F00D1124EC5FFD4F6181651306C06081BE
:10186000641303C06281E6120FC001968770D5CF62
:101870009F7011F0882331F3805E883018F3C8011F
:101880000E946309FD2CB1CFEE2009F4AECF809108
:101890003902816080933902F12CA7CF251306C04D
:1018A000941304C0F801EE2009F487C0C8010E9417
:1018B000BF09882319F1EE2009F1809139028032A5
:1018C00070F0209134023091350238872F831986C9
:1018D000BB86AA868C87CE0107960E94630986E0A4
:1018E000F801A4E3B2E001900D928A95E1F70E941D
:1018F000500B0E94410BFF24F39477CFC8010E9444
:101900006309F9CF311113C07A2DB98AA88A6E2DD7
:1019100089890E94C70984E392E00E94630986E0F6
:10192000F60111928A95E9F70E94410BB5CF251374
:101930000FC094130DC0E1100BC0F8018583C801DE
:101940000E94630986E0F60111928A95E9F74DCF6E
:10195000C8010E94BF09882389F2EE2079F28091A4
:101960003902803208F4BBCF209134023091350225
:101970003A8329831B82BD82AC828E83CE0101967D
:10198000ACCFE83CF10508F03EC0FE2CEE2009F497
:10199000B5CF25132AC0941328C08091390280FD49
:1019A0001BC0982F907FC1F0F8018583903F31F0E4
:1019B000982F907F905F8F70892B8583C8010E943C
:1019C000630986E0F801A4E3B2E001900D928A95E4
:1019D000E1F70E94410B09CF86E0F801A4E3B2E0F1
:1019E00001900D928A95E1F700CFC8010E94BF09CE
:1019F000811175CF80913902816080933902C801CD
:101A00000E946309F2CE7A2DB98AA88A6E2D89893F
:101A10000E94C70986E0F60111928A95E9F7D9CFAD
:101A2000EE2009F46BCFC8010E94BF09F82E88236D
:101A300009F464CF86E0F801A4E3B2E001900D92CE
:101A40008A95E1F784E392E00E9454060E94500BCD
:101A5000C0CF81E08E25D7CEACE0B0E0E2E3FDE080
:101A60000C94402C4F83588769877A878B879C8793
:101A7000CE0107960E94A50B882369F08A859B8575
:101A8000892B39F04F815885842F85238F3F09F0AA
:101A90006BC016E05FC086E0FE013796DE0111964E
:101AA00001900D928A95E1F78A859B85892B89F3B0
:101AB0008F81988589238F3F61F32091030230E065
:101AC000C9010196877099274091020248171906AB
:101AD00071F40E949F09109203021092020286E0A4
:101AE000E4E3F2E0DF011D928A95E9F7D2CF96E0B8
:101AF000929FD001939FB00D1124AC5FBD4FFE01AA
:101B0000319601900D929A95E1F7809303020E941D
:101B1000200BBFCF819FC00111248C5F9D4F0E947D
:101B2000A50B8823E9F0E09102021E9FF001112429
:101B3000EC5FFD4F40815181628173818481958189
:101B40000E94D1098091020290E001968770992746
:101B50008093020280910202909103028913DACFEE
:101B60002C96E3E00C945C2C69857A858B859C85AA
:101B70000E94D1098ECF682F8091040190910501B8
:101B80000E94E0220895682F809104019091050140
:101B90000E94EE22089580910401909105010E9417
:101BA000FC22089580915A02859585958595089522
:101BB00080915A028770089590915A02977081E03F
:101BC00009F480E0089580917D02089590917D024E
:101BD000892B80937D020895809590917D029823B2
:101BE00090937D02089510927D02089590917C0259
:101BF000892B80937C020895809590917C02982394
:101C000090937C02089510927C02089580915B026B
:101C1000089508950E94090E089590914F0392FF30
:101C200008C090915B02981721F080935B020E949C
:101C30000A0E089580915B02882329F010925B02BE
:101C400080E00E940A0E0895CF93DF93E091040193
:101C5000F091050180917D028083E0910401F09173
:101C60000501808190917C02892B808390915B0299
:101C7000992381F0E0910401F09105018081892B85
:101C8000808380910401909105010E944C22811172
:101C90000E941A0EC0910401D091050140E250E06B
:101CA0006AE372E0CE010E94D12C892B59F080E2C8
:101CB000FE01AAE3B2E001900D928A95E1F7CE0110
:101CC0000E940622DF91CF91089508950E94650E2B
:101CD000089590914F0392FF11C098E0899F900161
:101CE0001124622B60935A020E94160A80915A02B4
:101CF0008595859585950E94660E08950E94160A21
:101D0000089510925A0280E00E94660E0895909104
:101D10005A028095892380935A02282F277091F4C4
:101D2000282F082E000C330B9217130659F09091B0
:101D30004F0392FF07C08595859585950E94220ADD
:101D40000E94810E089590914F0392FB222720F963
:101D5000281769F080FB92F990934F0380914E030E
:101D600090914F030E94F50E82E00E94870E089525
:101D700080914F0382FB882780F991E089270E9498
:101D8000A30E089581E00E94A30E089580E00E94B2
:101D9000A30E08956FEF7FEF90E080E00E94102D7A
:101DA000089590E080E00E94EC2C883E9E4F19F44C
:101DB0000E94F61B089580E0089582E090E00E9462
:101DC000DE2C089583E090E00E94DE2C0895CF93EE
:101DD00084E090E00E94DE2CC82F82E290E00E9416
:101DE000DE2C982F8C2FCF910895CF93C92F682F79
:101DF00084E090E00E94F22C6C2F82E290E00E943E
:101E0000F22CCF910895AB01BC018FE090E00E94CD
:101E1000042D0895AB01BC0183E190E00E94042DE4
:101E2000089560E070E0CB010E940A0F089560E021
:101E300070E0CB010E94030F0E94110F089568EE1D
:101E40007EEF90E080E00E94102D60E082E090E064
:101E50000E94F22C60E083E090E00E94F22C10924D
:101E6000010260E084E090E00E94F22C64E082E2F3
:101E700090E00E94F22C60E085E090E00E94F22C5D
:101E800060E086E090E00E94F22C6FEF87E090E047
:101E90000E94F22C40E050E0BA0188E090E00E94FD
:101EA000042D60E08DE090E00E94F22C40E050E0D4
:101EB000BA0188E190E00E94042D60E087E190E0A3
:101EC0000E94F22C40E050E0BA018CE190E00E94C8
:101ED000042D70E060E080E290E00E94102D40E070
:101EE00050E0BA0188E190E00E94042D80E00E9459
:101EF0000F1C0E943E1C0E94170F08950E941F0F86
:101F00000895682F8EE090E00E94F22C08950E94C0
:101F1000C02360938E0270938F02809390029093FF
:101F2000910260938A0270938B0280938C0290934B
:101F30008D020895089508950E949B0F08950895B5
:101F40000E949F0F089584E192E10E94EF210E9478
:101F50009A0F0E949C0F089581E008950E94AC0F93
:101F60000895089508950E94B10F0E94B20F089538
:101F70000E9430120E94010608950E94AB230E9425
:101F80004E1C0E9408130E94B80F0E94011A0E9462
:101F9000A00F0895AAE0B0E0E0EDFFE00C94362C2D
:101FA0000E941E13A82E81110E94870F5EE7852EC6
:101FB00052E0952E10E000E0702E802F0E94531208
:101FC0006C01F401E190F1904F01E816F90609F473
:101FD00044C08091920281FD0E945C12C7018C2551
:101FE0009D25B12CEE24E394F12C9C012E213F2160
:101FF000232B69F10E94AE0F8823B1F0BE827F824D
:10200000CE20DF2081E0C114D10409F480E088876C
:102010000E94B4238160782F9A8789874E815F81DF
:1020200068858A850E941F06000F111FF801E2587B
:10203000FD4F80819181E826F926F182E08281E0DE
:10204000A11001C080E02A96EDE00C94522CB394CC
:10205000EE0CFF1CF0E1BF12C8CF0F5F1F4F063020
:10206000110509F0A9CF8FEF89838A831B820E9413
:10207000B4238160782F9D838C8349815A816B8141
:102080008D810E941F06DBCF0E94CA0F0E94471A53
:102090000E9414060895CF93DF930E943A11EC0139
:1020A000811522E59207E8F5811531E5930708F0DF
:1020B000ACC0883E910510F5803E910570F5883AD8
:1020C000910570F4853A910508F078C0813091054A
:1020D00021F1009711F1049700F5D0E0C0E01DC098
:1020E0008F3B9105D0F7C85AD0E0CC0FDD1FC95AFD
:1020F000DE4F0990D881C02DD4640FC0811540E512
:10210000940708F066C0C11580E4D80708F05EC0E7
:10211000CE019A9581159F4100F7CE01DF91CF91B5
:102120000895811536E5930718F5811545E594075F
:1021300008F083C0C11584E5D80708F079C09C2F4A
:10214000969596959E0123703327C115D34508F4C3
:1021500061C0C1E0D0E002C0CC0FDD1F2A95E2F7DC
:1021600030E2939FC0011124C82BD92BDA68D5CF58
:10217000C1158AE5D80778F4C11599E5D90708F0A3
:1021800066C0C11528E5D20708F4A7CFDC2FCC27FD
:10219000C06FD06AC2CFCE0190568115904208F030
:1021A0009CCF8D2F8F710E94D11190E0982F88279E
:1021B00088279F719C012C2BE90147C0C55AD0E0AC
:1021C000CB57DE4FC881D0E0D064A7CFDF70D06A94
:1021D000A4CFE4E096958795EA95E1F783702C2FDC
:1021E00026952695237040E2249F90011124382BD8
:1021F0008C2F8370C1E0D0E002C0CC0FDD1F8A9528
:10220000E2F7C22BD32BDC6888CFD82FCC27C16F45
:10221000D06A83CFC1E0D0E002C0CC0FDD1F2A9589
:10222000E2F720E2929FC0011124C82BD92BEBCFFB
:10223000DC2FCC27C46FD06A70CF0E94D111C82F79
:10224000D0E0DC2FCC27CC27DF71D06266CF8C2F7B
:102250008F700E94D11134E0D695C7953A95E1F779
:10226000CF709C2FEC01D06958CF0E945A200E9459
:102270004B10089582389105B1F1B0F48133910586
:1022800009F475C048F48932910509F469C08A32AD
:10229000910509F473C008958533910509F459C077
:1022A0008933910501F10895833E9105A9F138F430
:1022B000803E9105F9F0823E910549F10895863EF0
:1022C0009105A9F1873E9105C9F1843E910519F563
:1022D00020914F0321FF1FC080914E0384FD14C045
:1022E00087EE90E0089520914E032370A1F080EED8
:1022F00090E0089520914E0320FD47C030914F0398
:1023000030FF09C024FF44C090E080E004C0209169
:102310004E0322FDF7CF089520914E0322FD3BC0CE
:1023200030914F0330FDE3CF24FFF5CFEDCF209167
:102330004E0323FFF0CF24FDE7CFD2CF20914E03F1
:1023400023FD2CC030914F0331FFEECF84EE90E09F
:10235000089520914E0325FFDECF89E290E0089595
:1023600020914E0325FFD7CF85E390E0089520917B
:102370004E0326FFD0CF8AE290E0089520914E03CD
:1023800026FFC9CF81E390E0089589E390E00895A6
:1023900083EE90E0089582EE90E0089586EE90E05E
:1023A000089590914E0392FF06C0282F287128307F
:1023B000F9F4877F846093FF06C0282F28712831A5
:1023C000F1F4877E846120914F0320FF06C0382FEF
:1023D00038713830D9F4877F816021FF06C0282FFB
:1023E00028712831D1F4877E816194FD877E08951C
:1023F000282F24712430F9F68B7F8860DCCF282FBA
:102400002471243101F78B7E8861DDCF382F317143
:10241000313019F78E7F8860E0CF282F217121316C
:1024200021F78E7E8861E1CF80E008950E94CA0E78
:1024300008950E941E138FE39CE90197F1F700C0F5
:1024400000000E941E1380E00E94531280FF04C00F
:102450000E9416120E94FF2308950E9419120895E7
:102460000E94D10E811102C00E947E0F0E94DD0EDB
:10247000809392020E94E70E90934F0380934E0345
:102480000E942D120E94E20E0E94E7098091000234
:102490000E94FF09089508950E944B12089508951F
:1024A0000E944F120895E82FF0E0EE0FFF1FE45A4C
:1024B000FC4F808191810895089580EA8A95F1F713
:1024C000089500C008950E945D120895F894E82FC1
:1024D000E295EF70F0E031A1282F2F7081E090E0BD
:1024E00001C0880F2A95EAF7982F9095932391A31E
:1024F00092A1892B82A378940895CF93DF93C8E9A2
:10250000D1E089918F3F11F00E94661281E0CE39AF
:10251000D807B9F7C8E8D1E089918F3F11F00E9440
:10252000661281E0C839D807B9F7DF91CF910895D5
:10253000AF92BF92DF92EF92FF920F931F93CF93D0
:10254000DF938C01D62EC62FD0E0CE0188569E4F49
:102550007C01FC0120812F3F09F44DC0F894E22F4B
:10256000E295EF70F0E031A12F7081E090E001C0C2
:10257000880F2A95EAF7932F982B91A392A1809523
:10258000892382A378940E946112E8E8F1E048E987
:1025900051E021E030E0B12CA12C61916F3FA9F115
:1025A000A62FA295AF70B0E090968C9190E06F70DE
:1025B00002C0959587956A95E2F780FD26C0C9010E
:1025C000A82AB92A220F331F4E175F0731F7F701E8
:1025D00080818F3F11F00E94661261E0A114B10466
:1025E00009F460E08D2D0E946312CC0FDD1FC00F37
:1025F000D11FB982A882DF91CF911F910F91FF90D7
:10260000EF90DF90BF90AF90089590E080E0D8CF3A
:102610000E947D128CE0ECE5F3E0DF01982F1D9223
:102620009A95E9F7E0E5F3E0DF011D928A95E9F775
:1026300086E00E945A130E94A4040895ACE0B0E022
:10264000E4E2F3E10C943E2C8E010F5F1F4F8CE00F
:10265000F80111928A95E9F7F12C6F2DC8010E94BB
:102660009812F394F6E0FF12F8CF4CE050E0B80176
:1026700080E593E00E94D12CFF24F394009709F4A5
:10268000F12C892B41F08CE0F801A0E5B3E001903A
:102690000D928A95E1F72F2D46E06CE573E080E519
:1026A00093E00E945B130E94A7048F2D2C96E5E017
:1026B0000C945A2C0895FF920F931F93CF93DF939E
:1026C000F82E092F162FD72FC42F222349F081E08F
:1026D000809395020E94B423909394028093930276
:1026E000809195028823A1F08091930290919402A9
:1026F0000E94CC23059760F0EF2DF02FA12FBD2F66
:1027000090E080E0D0E08C179D073CF0109295029D
:10271000CDB7DEB7E5E00C945A2C219131912D9381
:102720003D930196F0CF0E94EE250E94BD0F0E94BE
:10273000FB2508950E9400260E9444100E941A263C
:1027400008950E944D230E94D4250E94A30F0E9449
:1027500093130E949A130E94B30FFBCFEF92FF9244
:102760000F931F93CF93DF93EB01E82FD1110EC08E
:10277000442321F0F0E0EA58FA4FE4916E2F7E2FC7
:102780008E2FCDB7DEB7E6E00C94592C0D2F10E05C
:10279000282F30E0442329F02A583A4FF901249198
:1027A00030E0F6E0CF9FC0011124EFEFF0E0BF0171
:1027B0000E94A92BAB018C2F90E0880F991FA5E5F3
:1027C000A49FB001A59F700D1124861B970B982F15
:1027D000990F980FBF01601B710B629FD001639F1F
:1027E000B00D729FB00D11248B2F9D9FB00111244D
:1027F000672F7727EF01C61BD70BBE01629FE00151
:10280000639FD00D729FD00D11247F01E91AF1084A
:10281000E09EB001E19E700DF09E700D1124672FB7
:102820007727E61BF70BE29F8001E39F100DF29FD5
:10283000100D1124E12F722F4230510599F048F408
:102840004115510569F04130510581F0EB2F8D2F75
:1028500007C04430510569F080F046305105B1F7AA
:102860006E2F8FCFE22F7B2F812FFACFE22F7D2F7C
:10287000F7CFEB2F822F712FF3CF7B2F822FED2FEE
:10288000EFCF41E00E94AE13089508950E944114D5
:102890000895CF93DF93762FE901682F842F0E944C
:1028A0004614798368838A83DF91CF910895403BF2
:1028B00008F04FEA0E944914089580916803982F08
:1028C0009E7F61F4817082608093680380916B03C6
:1028D000803B18F08FEA80936B0308958635B0F340
:1028E00081708465F1CF88E090E00E94E62C089525
:1028F000CF92DF92EF92FF926B017C010E945D14F8
:10290000B701A60188E090E00E94042DFF90EF90AF
:10291000DF90CF9008956091680370916903809172
:102920006A0390916B030E9478140895E8E6F3E03F
:1029300083E0808311828FEF82838FEA8383148206
:1029400060817181828193810E94781408958091C1
:10295000680380FF02C08695089580E008959091F5
:102960006C03933018F49F5F90936C03882351F0AD
:10297000609168037091690380916A0390916B0381
:102980000E947814089581E00E94AF1408959091F8
:102990006C03992319F0915090936C03882351F0A4
:1029A000609168037091690380916A0390916B0351
:1029B0000E947814089581E00E94C71408958091C0
:1029C0006C03089580936C03662351F06091680353
:1029D0007091690380916A0390916B030E9478144F
:1029E000089560E00E94E2140895809169030895BB
:1029F00080916A03089580916B03089570E00E94AE
:102A0000CA1B089560910A018091680380FF0BC082
:102A10008091090123E0829FC001112483599C4FBA
:102A20000E94FE14089580910B0190910C0123E007
:102A3000829FF0011124E359FC4F891748F7118256
:102A4000108212828F5F3396F8CF9091680390FFC7
:102A50000EC090910B0120910C0133E0939FF00187
:102A60001124E359FC4F921718F00E9402150895A3
:102A70008183608342839F5F3396F5CFA3E0B0E00C
:102A8000E4E4F5E10C94412C9091680390FF0AC0B6
:102A90009E012F5F3F4F0E9457144B8169818A81AD
:102AA0000E9425152396E2E00C945D2CCF93DF93D2
:102AB000EC01EC81F0E0EF58FB4F4491E8E6F3E0E5
:102AC000628181810E943E158C818F5F8C83DF91B2
:102AD000CF910895CF93DF93EC01E8E6F3E04381D3
:102AE00062818C810E943E158C818F5F8C83DF9187
:102AF000CF910895A3E0B0E0E0E8F5E10C943F2C1D
:102B00008C018091960281110AC09E012F5F3F4F78
:102B10004FEA6FEF0E9457148A8180939602F80162
:102B20006481613069F08091960240E0662361F033
:102B300040E0623011F44091960280E060E004C011
:102B40006091960240E080E00E942515F8018481A2
:102B500090E0019663E070E00E94BD2B8483239691
:102B6000E4E00C945B2CA3E0B0E0E9EBF5E10C941D
:102B70003A2C082FD62EE42EC22E9091680390FF97
:102B800029C0E92FE695AE2FB0E0A256BE4F8C913A
:102B900080931A039E7F923009F59E012F5F3F4F6D
:102BA000802F0E9457144B8169818A810E942515CC
:102BB00000936903D0926A03E0926B03CC2051F03A
:102BC000609168037091690380916A0390916B032F
:102BD0000E9478142396E9E00C94562C823019F464
:102BE000E0906B03E5CF863019F400916903E0CFE4
:102BF0008930D9F38931E1F6E9516E2F6170B62E33
:102C0000E695F0E0EF58FA4F1491F12C60910D0128
:102C1000F61618F00E940215CBCFF19EC0011124C8
:102C200070E00E94A92B802FB11014C0860F209154
:102C30000B01622F6F0D7727771F9B01220F331F28
:102C4000260F371F23593C4F4E2D6D2D0E945714D0
:102C5000F394DCCF861BEBCFE8E6F3E09181282FDD
:102C60004381628188E0890F0E94B315089581E055
:102C70000E942C160895E8E6F3E09181282F438105
:102C8000628188EF890F0E94B315089581E00E9448
:102C90003B160895E8E6F3E0628128E0620F08F44D
:102CA0006FEF282F438181810E94B315089581E041
:102CB0000E944A160895E8E6F3E0628128E0621B6C
:102CC00008F460E0282F438181810E94B3150895A4
:102CD00081E00E945B160895E8E6F3E0438128E076
:102CE000420F08F44FEF282F628181810E94B315B3
:102CF000089581E00E946C160895E8E6F3E04381B0
:102D000028E0421B08F440E0282F628181810E9464
:102D1000B315089581E00E947D16089520E00E9479
:102D2000B3150895EF92FF921F93CF93DF93EC01B9
:102D300010E0EE24EA94F12C60910D01161770F06A
:102D40000E9402159A818C8190FF27C08F5F8C832F
:102D5000DF91CF911F91FF90EF90089520910B018B
:102D6000422F410F5527551FCA019A01220F331FC9
:102D7000280F391F23593C4F70E0C7010E94BD2B1B
:102D8000962F8C8140916B0360916A03199F800D8F
:102D900011240E9457141F5FCFCF8150D8CFB0E0CD
:102DA000A0E0E5EDF6E10C94392CFC0182810FEFF7
:102DB00080FF01E010E048E1A42E80910D0118177A
:102DC00098F00E94021580919802013009F04FC0DE
:102DD000811102C080910D01815080939802CDB77E
:102DE000DEB7EAE00C94552CC0910B01C12ED12C1A
:102DF000CC0DDD2DD11DCE01880F991FC80FD91F15
:102E0000C359DC4F198218821A8234E0E32EF12C68
:102E1000B12C809198028B0D89311CF16A2D0E9492
:102E20009B2B892F082E000C990BC816D90691F4FC
:102E300080916B038E9DA0018F9D500D112455959F
:102E40004795559547959E0160916A038091690366
:102E50000E945714B00EF1E0EF1AF108D1F61F5F8F
:102E6000ACCF87FFDFCF90910D01890FDBCF90E0D2
:102E7000019660910D0170E00E94BD2BAECF0F93C3
:102E80001F93CF93DF9380910B0190910C0123E06E
:102E9000829FF0011124E359FC4F891740F1C0E0F3
:102EA000D3E060910D01C61740F10E9402152091F8
:102EB000070180919702820F8093970290910801F9
:102EC000920F90930801191654F4082E000C990BD8
:102ED00040910D014150550B841795071CF0219529
:102EE00020930701DF91CF911F910F9108951182D7
:102EF000108212828F5F3396D0CF0C2F10E070E0DB
:102F0000C8010E94BD2B20910B01820F482F50E079
:102F100020919702022E000C330B02171307BCF00E
:102F200020910801022E000C330B201731077CF092
:102F30008D9F9001112423593C4F40916B03609168
:102F40006A03809169030E945714CF5FAACFFA01E8
:102F5000EE0FFF1FE40FF51FE359FC4F11821082A3
:102F60001282F3CFB0E0A0E0E8EBF7E10C94372C4D
:102F7000EC014C81042F10E09801D8010E94082C2C
:102F80009B01AC010E941E2C4B015C01E0E2F0E0D1
:102F9000E01BF10BA5E5B0E0AC019B010E941E2CEB
:102FA0006B017C019F01DF010E94002C9B01AC01A1
:102FB0000E94292C9B01AC01280D391D4A1D5B1D67
:102FC000C701B6010E94D12BF22E822F90E039E288
:102FD0003F1520F143E0249F90011124359527955A
:102FE000122F109500E085E5E82EEF1880910D0175
:102FF000081718F10E9402159C8181E0992319F0AD
:10300000903219F48FEF8093060180910601890FA9
:103010008C83CDB7DEB7ECE00C94532C25E530E083
:10302000B901681B790B9B01220F331F260F371F35
:1030300037FFD4CF2F5F3F4FD1CF8E2D01FD8F2D86
:1030400020910B01622F600F7727771F9B01220FC2
:10305000331F260F371F23593C4F412F60916A03BE
:103060000E9457140F5FC2CF0F931F93CF93DF932C
:10307000EC0110E000E090910D019017110609F0AD
:103080006CF40E9402158C8190E001968170992762
:103090008C83DF91CF911F910F91089520910B01A7
:1030A000A801420F511D9A01220F331F240F351F13
:1030B00023593C4F4C8160916A0380916903969536
:1030C0009017110651F04CF0442349F040916B03E6
:1030D0000E9457140F5F1F4FCECF4423B9F340E037
:1030E000F7CFB0E0A0E0E7E7F8E10C94332CFC0167
:1030F0006280448081E08483E1E7F4E07490E0EF53
:10310000F4E0E491812C75E0972EF2E0CF2EDD24DF
:10311000D394AA24AA94B12C55245A94E7190E2FBB
:1031200010E080910D01881638F00E940215CDB78D
:10313000DEB7E0E10C944F2CE82CF12C82E08615F0
:1031400068F09E9CF0019F9CF00D1124E756FD4F06
:1031500080916903808380916A038183411023C039
:103160009E9CF0019F9CF00D1124E756FD4F1382A9
:10317000128220910B01C701820F911D9C01220F29
:10318000331F280F391F23593C4F9E9CF0019F9CF1
:10319000F00D1124E756FD4F4281618180810E942C
:1031A00057148394BECF9E9CE0019F9CD00D1124A8
:1031B000C756DD4F8B818823E9F081508B83859D35
:1031C000C00111246C8170E00E94A92BFB01FF2734
:1031D000EF58FB4F8491E82FE719E59DC0011124BA
:1031E000B8010E94A92B80916B03689FB001112444
:1031F0007A83BFCF0E94B42C20916B03269521586F
:103200002C9DA0012D9D500D1124452F552784176D
:1032100095070CF0AECF82E0861588F40E94B42C9E
:10322000B5010E94BD2B88830E94B42C20916A03B3
:103230002695622F70E00E94BD2B280F29839E9C4B
:10324000F0019F9CF00D1124E756FD4F12828091F2
:103250006B03893C58F088EC9E9CF0019F9CF00D1C
:103260001124E756FD4F8483838383CF8431A0F7F5
:1032700084E1F2CFE8E6F3E080818E7F8083608195
:103280007181828193810E94781410921B032FEF29
:1032900080E792E0215080409040E1F700C00000BC
:1032A0000E9402150895E8E6F3E080818E7F808316
:1032B00010921B032FEF80E792E021508040904056
:1032C000E1F700C000000E940215089510921B0350
:1032D0008091180381110AC081E0809318038091C6
:1032E00068038170809317030E94531908956091B9
:1032F0006803669570E04BE050E08EE091E00E943C
:10330000C42C892B19F481E080931B030E94B42301
:10331000909312038093110308959091680390FF96
:103320002BC09170811129C092609093680366232D
:1033300051F0609168037091690380916A039091E4
:103340006B030E94781460916803669570E04BE00F
:1033500050E08EE091E00E94C42C892BA9F01092DD
:103360001B0381E08093140340916B0360916A0317
:10337000809169030E948E1608958B3210F0946537
:10338000D4CF880F982BD1CF0E947719EACF682F1E
:1033900090916803969581E0890F8B3208F081E067
:1033A0000E948D19089581E00E94C7190895682F21
:1033B0009091680396958FEF890F09F48AE20E9435
:1033C0008D19089581E00E94D719089561E00E9447
:1033D0008D190895E8E6F3E0808181608083869509
:1033E0000E94E61908958091680380FF03C00E943F
:1033F0003A1908950E94EA19089560E00E948D1913
:1034000008958091190381112EC00E94D10E81115F
:1034100004C00E947E0F0E9496140E947314609351
:1034200068037093690380936A0390936B036E7FC4
:1034300061F40E9496140E94731460936803709361
:10344000690380936A0390936B030E945D1410924A
:103450001B038091680380FF03C086950E94FD19BD
:1034600081E0809319030895E8E6F3E080818160AC
:10347000808386950E94FD1908951092180380910B
:10348000170381110E94341A0E94771908950F932F
:103490001F93CF93DF9380911B038823B9F1809111
:1034A0001A03E0916803E695E81BE093130382306A
:1034B00091F5F0E0E359FB4FE491CE2FD0E006E523
:1034C00015E180911403882361F0109214030E9487
:1034D000B423909312038093110310921603109259
:1034E00015030E94B423E0911103F09112038E1B87
:1034F0009F0B8F3F9F4750F4EC0FFD1FF09312037B
:10350000E093110381E193E0F8010995DF91CF91F8
:103510001F910F910895863049F4F0E0E659FB4F72
:10352000E491CE2FD0E00AE615E1CBCF893051F4FB
:10353000E695F0E0E959FB4FE491CE2FD0E002E9A7
:1035400016E1BFCF8F3051F4E695F0E0EC59FB4F18
:10355000E491CE2FD0E00FEC16E1B3CF853149F4E2
:10356000F0E0EF59FB4FE491CE2FD0E00FE317E1ED
:10357000A8CFC8E2D0E002EB17E1883109F4A1CF6F
:10358000833239F4EFE5F4E0C591D4910AE715E10F
:1035900098CFC4EFD1E004E318E1843209F491CF6D
:1035A000C0EDD7E005E414E1853209F08ACF8E2F13
:1035B00063E00E948F2BE92FF0E0E45AFB4FE49187
:1035C000CE2FD0E001E718E17CCFFA01811101C0D4
:1035D000FB0109950895CF93DF93C82FD62F0E9442
:1035E000A7148C1748F00E94A7148D1728F40E9486
:1035F000D319DF91CF9108958C2F0E94E619F9CF4E
:103600001F93CF93DF93EC01FB01128111111BC0BB
:103610000E94E30D8272CC3CFCE5DF0709F4A0C0F8
:1036200008F045C0C63CECE5DE0709F485C0F8F4B7
:10363000C33C9CE5D90709F475C050F4C23CDC4595
:1036400009F46DC011E0812FDF91CF911F91089592
:10365000C43C9CE5D90709F46AC046E456E167E337
:1036600076E1C53CDC4571F70E94E51AECCFC93C18
:10367000FCE5DF0709F46AC068F4C73CECE5DE0747
:1036800009F45FC047E556E168E676E1C83CDC45F1
:1036900059F3D8CFCA3C9CE5D90709F45CC04BED7F
:1036A00054E163EC74E1CB3CDC45F1F2CBCFC13D9E
:1036B000FCE5DF0709F463C098F4CE3C9CE5D9072C
:1036C00009F457C008F451C0CF3CFCE5DF0709F40A
:1036D00053C0C03DDC4509F0B5CF6EE089E01CC0A9
:1036E000C43D9CE5D90709F450C058F4C23DFCE53F
:1036F000DF0709F447C0C33DDC4509F0A3CF88E1EB
:1037000035C0C53D9CE5D90709F442C06AE285E2AF
:10371000CD35DD4509F096CF0E94EB1A94CF0E947B
:10372000F31991CF42EE59E163ED79E19DCF43ED7D
:1037300059E162EE79E198CF47E356E166E476E13C
:1037400093CF48E656E167E576E18ECF4AE856E149
:1037500069E776E189CF49E756E16AE876E184CF07
:1037600043EC54E16BED74E17FCF81E00E94E619F8
:103770006ACF65E082E0D0CF68E086E0CDCF64E13B
:103780008FE0CACF67E185E1C7CF62E289E1C4CFAC
:1037900083E2ECCF279A45B14F7755B15068EFB728
:1037A000F8949B01220F331F260F371F280F391F54
:1037B0002817390741F4EFBF8FE594E00197F1F73F
:1037C00000C000000895DC016D91CD0178E055B98D
:1037D000000000C067FF45B9660F000000C000C0D0
:1037E00000C045B900C07A9591F7E2CF83E290E03E
:1037F0000E94DE2C823289F484E290E00E94DE2C6A
:10380000863059F485E290E00E94DE2C91E0873109
:1038100009F090E0892F8170089580E0FCCFCF936C
:10382000C82F6FEF811162E283E290E00E94F22CD8
:103830006FEFC11166E084E290E00E94F22C6FEF1E
:10384000C11167E185E290E00E94F22CCF910895CA
:10385000089586E290E00E94DE2C682F70E090E0F0
:1038600080E008950895CF93C62F0E94321C6C2FDC
:1038700086E290E00E94F22CCF91089580E00E94B1
:103880000F1C60E070E0CB010E94331C0E94DA1F25
:103890000E94B52081E00E940F1C08950E94281C00
:1038A0000E94291C0E94321C0E94F61B811102C03A
:1038B0000E943E1C0895CF93FB01C281CC2309F1E5
:1038C0009C0122513F452031310520F582510E9453
:1038D000C520C0E08C2FCF91089581E00E94160A88
:1038E00043E062E081E00E949A04F3CF81E00E940D
:1038F000220A43E062E081E00E949A04EBCF82E07A
:10390000F6CF8031FFE59F0789F381319F45B9F3F9
:10391000C1E0E0CF8031EFE59E07F9F281319F45AC
:10392000C9F682E0DBCF2FEFFC0120830895CF930F
:10393000DF93EC0188818138A9F028F4803871F098
:10394000DF91CF910895823881F08338C9F70E94C2
:10395000F51489830E94F8148A83F2CF0E94FB1425
:103960008983EECF0E94A714FBCF0E94DF14F8CF0B
:10397000CF93DF93EC0188818138D9F028F4803827
:1039800069F0DF91CF9108958238F9F08338C9F753
:103990000E94FB14482F6A81898108C0D9810E9446
:1039A000F814C82F0E94F5144D2F6C2F0E948E160C
:1039B000E8CF89810E94FD198981811103C00E948D
:1039C0005319DFCF0E94341ADCCF89810E94F11491
:1039D000D8CFEF92FF920F931F93CF93DF93EC0119
:1039E000062FDC01ED91CD01E150E33108F0ACC0D0
:1039F000F0E0ED5AF24D0C94F32B198289E08A83A2
:103A0000602FCE010E94A724CDB7DEB7E6E00C946C
:103A1000592C8981823069F0833071F08130D9F47A
:103A20000E94C0230E94F92B6A837B838C839D8331
:103A3000E7CF0E94291CF6CF7E0110E0812F0E9463
:103A40005312F701928383831F5FF2E0EF0EF11CA4
:103A50001630A1F7D5CF602FCE010E94931CD0CF96
:103A600089818230C1F76A817B818C819D810E942E
:103A7000F92B0E94331CC4CF4B816A8189810E943B
:103A80009C1F9827892798279D838C83B9CF2C81E9
:103A90003D813227232732274B816A8189810E9409
:103AA000BE1FAECF0E94DA1FABCF0E94B81CA8CFBA
:103AB0000E94971CA5CF0E948B14A2CF0E94682061
:103AC00089839ECF0E946A209827892798279A8306
:103AD000898396CF6B8170E089819A81AE014C5FBA
:103AE0005F4F9827892798270E946D2089CF6B8187
:103AF00070E089819A81AE014C5F5F4F98278927DA
:103B000098270E9491207CCF0E94B52079CF0E94F7
:103B1000891FD6CF6B8170E089819A81AE014C5F9D
:103B20005F4F9827892798270E94122069CF6B81C1
:103B300070E089819A81AE014C5F5F4F9827892799
:103B400098270E9436205CCF8FEF888359CFCF9380
:103B5000DF93EC01FB018281882309F433C1C33078
:103B6000FDE5DF07C0F5CA3F9CE5D90730F49E01AB
:103B700022503C4524313105B0F50E94E70E909368
:103B80004F0380934E03C1318CE5D80709F4EEC092
:103B900008F069C0C930ECE5DE0709F4D5C0C8F506
:103BA000C5308CE5D80709F4C7C000F5C330ECE593
:103BB000DE0709F4B9C008F0BBC0C230DC4509F427
:103BC000ADC080914E0390914F030E94F50E0E946C
:103BD0009F0980E008C0C136EDE5DE0771F2C53A05
:103BE000FDE5DF0751F2DF91CF91089580914E03FB
:103BF0008062C7309CE5D90709F493C080914E03D9
:103C00008061C830DC4508F48CC080914E0380642C
:103C100088C080914E038B7FCD30FCE5DF0709F42F
:103C200080C098F480914E038E7FCB309CE5D907FD
:103C300009F477C080914E038C60CC30DC4508F4E9
:103C400070C080914E038D7F6CC080914E038F7E3B
:103C5000CF30FCE5DF0709F464C008F47BC0809135
:103C60004E038F7D5EC0CD3F9CE5D90709F47AC035
:103C700050F5C531FCE5DF0709F486C098F4809162
:103C80004E03837FC3319CE5D90709F44AC008F489
:103C900071C00E949F0990914E03892F97FB87F96D
:103CA00080583FC0CB3FFCE5DF0709F449C008F06E
:103CB00055C080914F038160CA3FDC4509F081CF38
:103CC00080934F037ECFC130EDE5DE0709F468C075
:103CD000A8F4CF3F8CE5D80709F452C080914F0378
:103CE0008360C115DD4560F380914F03982F909557
:103CF00091708E7F892B90FB81F9E2CFC136EDE583
:103D0000DE0709F451C0C53AFDE5DF0709F453C0E9
:103D1000C230DD4509F055CF80E043C080914E03AD
:103D2000816080934E034DCF80914E038260F9CF26
:103D300080914E038460F5CF80914E038860F1CF6F
:103D400080914F038260BCCF0E949F0980914E03F7
:103D50008068E7CF80914E03877FE3CF80914F0348
:103D60008E7FAECF80914F038D7FAACF80914E037F
:103D70008F7BD7CF0E949F0980914E038F77D1CF41
:103D800080914F038C7F9CCF80914E0382FB9927BB
:103D900090F921E0922790FB82F990FB83F9C1CF43
:103DA00081E00E94810F0DCF90914E03892F8F7E6D
:103DB00094FF8061B6CF90914E03892F8E7F90FF44
:103DC0008160AFCF81E00FCFEBEFE80FEF3308F06A
:103DD00062C0F0E0EA59F24D0C94F32B0E947E0F82
:103DE00081E0089580919202807F8093920281E029
:103DF00080931C0308950E94B904F2CF909192021F
:103E0000892F8E7F90FF81608093920280FDE8CFA2
:103E1000817F80939202E4CF90919202892F8D7FCF
:103E200091FF82608093920281FFDACF80919202AB
:103E30008160EFCF90919202892F8B7F92FF8460F7
:103E40008093920282FDF2CFCBCF90919202892F84
:103E5000877F93FF88608093920283FDE7CFC0CF76
:103E60000E949F0990914E03892F97FB87F98058F4
:103E700080934E03B5CF81E00E94E7090E949F091D
:103E8000AFCF895391E001C0990F8A95EAF7892F46
:103E9000F3CF8D51F7CF80E0089580E008950E9420
:103EA0004D1F0895CF93C82F80911C03882331F0B4
:103EB000813099F010921C0380E00DC00E94E30D48
:103EC0008232D1F78C2F0E944D1F811116C08C2F8A
:103ED0000E94E41E8170CF9108950E94E30D82320A
:103EE00089F38C2F0E944F1F811105C0C43171F0DE
:103EF00038F4CB3079F781E0EDCF81E090E0EACF84
:103F0000C93221F0C833B9F380E0E4CF10921C032A
:103F1000FBCF84E0089590E2699FB001112450E046
:103F2000440F551F640F751F90EC899F600D711D24
:103F30001124CB01879608950F931F93CF93DF939E
:103F40008430C8F46630B8F44031A8F40E948B1F66
:103F50008C010E94DE2CC82FD0E0DC2FCC27C801BA
:103F600001960E94DE2C9E01282BC901DF91CF9182
:103F70001F910F91089590E080E0F8CF0F931F9369
:103F8000CF93DF93122F032F843078F4663068F4D8
:103F9000403158F40E948B1FEC01602F0E94F22CDC
:103FA000612FCE0101960E94F22CDF91CF911F91DB
:103FB0000F910895AF92BF92CF92DF92EF92FF924E
:103FC0001F93CF93DF938CEAC82E80E0D82ED0E0E9
:103FD0007601C0E014C0F50125913491412F6C2F7A
:103FE0008D2F0E94BE1F82E0A80EB11C1F5F1031F2
:103FF00091F780E2E80EF11CCF5FC63019F057014F
:1040000010E0E9CFDF5F80ECC80ED11CD43001F79F
:10401000DF91CF911F91FF90EF90DF90CF90BF90F5
:10402000AF900895EF92FF920F931F93CF93DF937A
:10403000EC018A017C01E60EF71ECE018796CE15B3
:10404000DF0529F4CDB7DEB7E6E00C94592CC11595
:1040500023E0D20740F40E94DE2CF80180830F5F3A
:104060001F4F2196EACFF8011082F9CFB0E0A0E00F
:10407000ECE3F0E20C943B2C7C016A018C01060F0E
:10408000171FEC01CE018796C017D10729F4CDB7D1
:10409000DEB7E8E00C94572CC11523E0D20740F4BA
:1040A000FE01EE19FF09EC0DFD1D60810E94F22C4E
:1040B0002196E8CF462F843040F4763030F46031DA
:1040C00020F4672F0E949C1F089590E080E00895DF
:1040D00080E1089589ED90E00895EF92FF920F93AB
:1040E0001F93CF93DF93EC018A017C01E60EF71E4C
:1040F000CE01895D9C4FCE15DF0529F4CDB7DEB723
:10410000E6E00C94592CC93DD10540F40E94DE2C08
:10411000F80180830F5F1F4F2196EACFF8011082CC
:10412000F9CFB0E0A0E0E7E9F0E20C943B2C7C0191
:104130006A018C01060F171FEC01CE01895D9C4FAF
:10414000C017D10729F4CDB7DEB7E8E00C94572C9F
:10415000C93DD10540F4FE01EE19FF09EC0DFD1D2E
:1041600060810E94F22C2196E8CFCF93DF93C7E2C3
:10417000D3E060E0CE010E94F22C2196C11584E0CC
:10418000D807B9F7DF91CF910895A4E0B0E0EBEC48
:10419000F0E20C943C2CF82E8FE08F1548F18FEF55
:1041A00093E00E94DE2C811123C007E213E0F1109E
:1041B00023C019821A821B821C82DD24D3947801C9
:1041C0008FEFE81AF80AC8010E94DE2C89831A8250
:1041D000882371F09FEF980F9330D8F48A83D982A7
:1041E0000E5F1F4FC7010E94DE2C8B83811112C00E
:1041F0002496E7E00C94582C011584E01807C1F3CD
:10420000C8010E94DE2C811101C0FA940F5F1F4F7C
:10421000CECF8701CE0101960E94F405D0CFCF9377
:10422000DF93EB0186319C4511F50E94E30D9A81E5
:10423000992399F08A7A91E009F490E090931D0314
:10424000811109C089E20E94BB0D0E94240E80E00A
:10425000DF91CF91089585E3F6CF80911D03811101
:1042600004C089E20E94C30DF0CF85E3FBCF81E05B
:10427000EFCF0F931F93CF93DF93C42FD22FFC0167
:1042800082818823C9F0409320030E94B423909335
:104290001F0380931E0380E28C0F883040F4C770A8
:1042A00081E001C0880FCA95EAF70E945A07DF91A2
:1042B000CF911F910F91089510912003141332C0D4
:1042C00080911E0390911F030E94CC23883C91058E
:1042D00048F5C0E2CD0F1D17B9F080E2810F88309C
:1042E00040F4177081E001C0880F1A95EAF70E9428
:1042F0006107C83048F481E09D2F977001C0880F96
:104300009A95EAF70E945A07802F0E945107C830F9
:1043100070F6D77081E001C0880FDA95EAF70E9445
:104320006107C5CF80E28C0F883008F6C77081E046
:1043300001C0880FCA95EAF7F2CF0F939C01CB0119
:10434000233F4CE5340759F1A8F4283DFCE53F072D
:1043500001F1293D4CE53407D1F1273D3C4591F46D
:1043600006E221EE41EE67ED7CE50E94392180E016
:104370000F910895253FFCE53F07E9F0B0F0263F97
:104380003C45F9F0FC018281882339F11092200329
:10439000EFCF07E225EE45EE68ED7CE5E6CF06E2DD
:1043A00021EE40EE63EF7CE5E0CF07E225EE44EE40
:1043B00064EF7CE5DACF06E221EE42EE65EF7CE5C4
:1043C000D4CF07E225EE46EE66EF7CE5CECF08E2DD
:1043D00021E045EE69ED7CE5C8CF81E0C9CF90933F
:1043E000D9018093D80108959093260380932503E3
:1043F0000895E0912503F0912603309729F001906C
:10440000F081E02D0995089580E00895E09125035D
:10441000F0912603309799F020912501222359F03D
:1044200020914E0327FF07C0DC012C9111962C939D
:10443000119726E02C930280F381E02D09950895D1
:1044400020912303309124032817390771F09093AA
:10445000240380932303E0912503F09126033097F2
:1044600021F00680F781E02D099508952091210320
:10447000309122032817390771F09093220380931B
:104480002103E0912503F0912603309721F0008469
:10449000F185E02D09950895FC0132968091250162
:1044A000882321F080914E039EE187FF96E080E013
:1044B000915008F4089521912223D1F38F5FF8CF12
:1044C000662301F1209125012223F1F020914E0372
:1044D00027FF1AC0462F4695469546954E3190F4D3
:1044E000677021E030E002C0220F331F6A95E2F7C7
:1044F000840F911DFC01828190E02823392381E003
:10450000232B69F480E00895FC01329608962191EE
:10451000261721F0E817F907D1F7F4CF81E00895C5
:104520009C01FC0132969FEF80E04191461751F0CB
:104530009F3F19F4411101C0982F8F5F8630A9F772
:104540009F3F09F40895290F311D97FD3A95F90110
:1045500062830895FC01329608962191261303C0C8
:10456000DF0111971C92E817F907B9F70895E62FB4
:10457000E695E695E695EE3168F4E80FF92FF11D22
:10458000677021E030E001C0220F6A95EAF782816E
:10459000822B82830895E62FE695E695E695EE3127
:1045A00070F4E80FF92FF11D677021E030E001C0D1
:1045B000220F6A95EAF720958281282322830895A5
:1045C00020912501222339F020914E0327FF03C0BB
:1045D0000E94B72208950E949022089520912501FB
:1045E000222339F020914E0327FF03C00E94CB22E3
:1045F00008950E94AA220895FC0132968091250117
:10460000882351F080914E0387FF06C08EE1DF01C1
:104610001D928A95E9F7089586E0F9CF08950E94E2
:104620000E230895811106C081E0809327030E9424
:104630000F23089582E0F9CF83E0809327030E943F
:104640000F2308950E941223089581E08093270389
:104650000E940F2308950E94252308950895089528
:104660000E942F230895089508950E942E230895EF
:10467000CF930E9433230E941E130E943423C0E074
:104680008C2F0E945312892B31F4CF5FC630C1F7B3
:1046900080E0CF91089581E0FCCF85B7806885BF29
:1046A00085B7806885BF08951F921FB61F92112499
:1046B0008F939F93AF93BF9380912803811113C071
:1046C0008091B5039091B603A091B703B091B80360
:1046D0004196A11DB11D8093B5039093B603A0939D
:1046E000B703B093B803BF91AF919F918F911F9083
:1046F0001FBE1F9018958091BD03843031F10E9438
:1047000023051092280388E190E020E40FB6F89486
:10471000A895809360000FBE2093600083B7817FCF
:10472000846083BF83B7816083BF7894889583B7A3
:104730008E7F83BF0FB6F894A89580916000886142
:1047400080936000109260000FBE08950E949F0940
:104750000E942A05089582E084BD93E095BD9AEFFA
:1047600097BD80936E0008952FB7F8948091B5039C
:104770009091B603A091B703B091B8032FBF0895ED
:104780002FB7F8946091B5037091B6038091B70389
:104790009091B8032FBF08959C014FB7F894809172
:1047A000B5039091B603A091B703B091B8034FBF82
:1047B000821B930B089578941F921FB61F921124A9
:1047C0008F939F93AF93BF938091B5039091B6035E
:1047D000A091B703B091B8030196A11DB11D8093BC
:1047E000B5039093B603A093B703B093B803BF91FA
:1047F000AF919F918F911F901FBE1F90189581E0E0
:104800008093E00080E28093D8001092C9008FE18D
:104810009EE40197F1F700C0000087E090EBDC0117
:104820008093C6039093C703A093C803B093C903B2
:1048300088E19CE00FB6F894A895809360000FBEC5
:1048400090936000FFCF88E19CE00FB6F894A895A4
:10485000809360000FBE90936000FFCF80914C0367
:1048600008950895CF93DF93EC018091250188236B
:10487000B1F180914E0387FF32C060E284E0809303
:10488000E9008FEF9091E800815095FD06C095ED0D
:104890009A95F1F700008111F5CF8091E80085FF2E
:1048A0001BC08091250170E050E040E0811104C000
:1048B00050E040E068E070E0CE010E94B9268091AF
:1048C000E8008E778093E80080E2FE01ACE2B3E07E
:1048D00001900D928A95E1F7DF91CF91089568E0FC
:1048E00081E0CDCF8093290370932B0360932A033B
:1048F0008091BD038430F9F48093E9008FEF9091AB
:10490000E800815095FD06C095ED9A95F1F70000FD
:104910008111F5CF8091E80085FF0DC050E040E0A7
:1049200063E070E089E293E00E94B9268091E8009C
:104930008E778093E8000895BC0184E00E94722481
:104940000895BC0183E00E94722408950895CF93D6
:10495000FC01603221F58091BD03843001F5C091E6
:10496000E900CF702091EC00922F917020FD90E82B
:10497000C92B82E08093E9008091E80080FF0CC0A1
:1049800050E040E060E270E0CF010E94B9268091E3
:10499000E8008E778093E800CF70C093E900CF9154
:1049A00008958091BC03811109C00E9498280E943B
:1049B000F5288091E20084608093E20008951092CF
:1049C000BC0308950E94252308956091B90381E0F6
:1049D000611101C080E00E941C2308959091BD03E5
:1049E00081E0943009F080E06091B9030E942223B5
:1049F000089542E061EC81E00E94142842E261ECFB
:104A000084E00E94142842E261EC82E00E941428B3
:104A100042E260EC83E00E9414289091BD0381E0A3
:104A2000943009F080E06091B9030E941223089548
:104A30008091BF03833009F463C030F48130E1F129
:104A4000823009F4A0C008958A3009F48CC08B30FC
:104A500009F471C0893009F052C08091BE038132DF
:104A600009F04DC08091C2039091C303009719F0E3
:104A7000029709F044C08091E800877F8093E800A6
:104A80008091E80082FF37C09091F3008091F2009E
:104A9000029731F48091F100813011F0863021F4D9
:104AA0008091F10080934C038091E8008B77809394
:104AB000E8000E94482823C08091BE03813AF9F49F
:104AC0008091E800877F8093E8008091C2039091F5
:104AD000C303892B61F460E28CE293E070E00E94F2
:104AE00057278091E8008B778093E800089560E075
:104AF00090E080E0F3CF8091BD038111C1CF089594
:104B00008091BE03813AD9F78091C2039091C3038B
:104B1000892BA9F78091E800877F8093E800809136
:104B2000E80080FFFCCF809125018093F100809107
:104B3000E8008E77BCCF8091BE03813201F780916F
:104B4000C2039091C303892BD1F68091E800877F3F
:104B50008093E8000E9448288091C003809325013B
:104B60000E949F0908958091BE03813241F6809191
:104B7000E800877F8093E8000E9448288091C10365
:104B800080934D0308958091BE03813A09F0B7CF19
:104B90008091E800877F8093E8008091E80080FFA3
:104BA000FCCF80914D03C1CF84B7877F84BF0FB600
:104BB000F894A895809160008861809360001092BD
:104BC00060000FBE80E890E00FB6F894809361001B
:104BD000909361000FBE0E942B2308950E94982895
:104BE0000E94F528E2EEF0E0808184608083789472
:104BF0000E94742B089589E191E00E94F4210895A8
:104C00008091BD03853031F48091BD03853019F06A
:104C10000E94A62308950E947B238091BB038823D2
:104C200099F30E943823882379F30E94A3260E94D7
:104C30009F09EACFA0E2B0E0E0E2F6E20C94412C5A
:104C40008091BD03843009F583E08093E900809171
:104C5000E80082FF1AC08091E80090E085FF09C05B
:104C600050E040E060E270E0CE0101960E9408272B
:104C700091E08091E8008B778093E800992329F0F8
:104C800060E2CE0101960E94E91CA096E2E00C943D
:104C90005D2C0E944C260895292F3327233031059F
:104CA00021F168F42130310509F443C02230310587
:104CB00009F444C090E080E030E020E026C02132DA
:104CC000310551F122323105A9F76330710590F7B2
:104CD000FB01EE0FFF1FE453FE4F2081318167532C
:104CE0007E4FFB01808190E010C0992781309105B3
:104CF00081F0009729F00297E9F6E6E7F6E002C0B6
:104D0000E8EAF6E0849190E09F01FA013183208384
:104D10000895EAE8F6E0F6CF6330710558F6660FBD
:104D2000771FFB01EE52FE4F2081318189E090E038
:104D3000ECCF82E190E027E037E0E7CF8BE590E031
:104D40002CEA36E0E2CF80E189BD82E189BD09B479
:104D500000FEFDCF8091D8008F7D8093D800809198
:104D6000E00082608093E0008091E00081FDFCCF54
:104D70000895AF92BF92CF92DF92FF920F931F934D
:104D8000CF93DF936C01EB018A010E946728F82E14
:104D9000811123C00115110539F0F801808191813D
:104DA000C81BD90BC80ED91EB12CA12C2097A9F075
:104DB0008091E80085FD22C08091E8008E77809385
:104DC000E80001151105A1F0F80180819181A80E7C
:104DD000B91EB182A08285E0F82E8F2DDF91CF9190
:104DE0001F910F91FF90DF90CF90BF90AF900895EB
:104DF0000E9467288823D1F2F82EEFCFF601819127
:104E00006F018093F1002197FFEFAF1ABF0ACECF59
:104E1000AF92BF92CF92DF92FF920F931F93CF93E7
:104E2000DF936C01EB018A010E946728F82E811143
:104E300023C00115110539F0F80180819181C81B4B
:104E4000D90BC80ED91EB12CA12C2097A9F08091A6
:104E5000E80085FD22C08091E8008B778093E80010
:104E600001151105A1F0F80180819181A80EB91EEC
:104E7000B182A08285E0F82E8F2DDF91CF911F9116
:104E80000F91FF90DF90CF90BF90AF9008950E9458
:104E900067288823D1F2F82EEFCF8091F100F60138
:104EA00081936F012197FFEFAF1ABF0ACECFFC01AC
:104EB0008091C4039091C50386179707A0F06115F0
:104EC000710529F49091E8009E779093E80090E0B6
:104ED0006115710551F4911108C08091E80082FFBD
:104EE00034C080E00895BC01F2CF8091BD038823D7
:104EF000C1F18530C1F18091E80083FD30C080911F
:104F0000E80082FDEACF8091E80080FFE1CF809148
:104F1000F3002091F200382F6115710519F0283047
:104F2000310558F091E02830310509F090E02091EA
:104F3000E8002E772093E800CBCF81918093F10099
:104F4000615071092F5F3F4FE7CF8091BD038823E8
:104F500041F0853041F08091E80083FFBECF81E0D1
:104F6000089582E0089583E00895FC018091C403D0
:104F70009091C50386179707A0F06115710529F474
:104F80008091E8008E778093E80090E061157105CC
:104F900051F4911108C08091E80082FF35C080E093
:104FA0000895BC01F2CF8091BD038823C9F18530FB
:104FB000C9F18091E80083FD31C08091E80082FD55
:104FC000EACF8091E80080FFE1CF8091F30020914B
:104FD000F200382F6115710519F02830310558F0AD
:104FE00091E02830310509F090E08091E8008E775B
:104FF0008093E800CBCF84918093F100319661508B
:1050000071092F5F3F4FE6CF8091BD03882341F0A8
:10501000853041F08091E80083FFBDCF81E00895A5
:1050200082E0089583E00895982F973028F08F70DC
:105030008093E90081E008959093E900242F762F72
:1050400050E0981731F07091EC002091ED005091F4
:10505000F00021FD02C09F5FE8CF3091EB003E7F62
:105060003093EB003091ED003D7F3093ED003091B7
:10507000EB0031603093EB007093EC002093ED0077
:105080005093F0002091EE0027FDE5CF80E00895D9
:105090008091BE0387FF13C08091E80082FF06C0A5
:1050A0008091E8008B778093E80004C08091BD0375
:1050B0008111F2CF08958091BD038823D9F38091A7
:1050C000E80080FFF8CF8091E8008E77ECCF209148
:1050D000E4003091E50095E6A9012091EC00822FD3
:1050E000817020FF06C08091E80080FF06C080E04C
:1050F00008952091E80022FD1AC08091BD03882305
:1051000089F0853089F08091EB0085FD0FC02091FA
:10511000E4003091E50042175307F9F29150E1F6AF
:1051200084E0089582E0089583E0089581E0089581
:105130000E9407290E940F29E0EEF0E08081816043
:105140008083E8EDF0E080818F77808319BCA7ED44
:10515000B0E08C918E7F8C9380818F7E80831092C3
:10516000BC0308950F931F93CF93DF930E940729E9
:105170000E940F29C8EDD0E088818F7788838881CD
:105180008068888388818F7D888319BC1092BD03D5
:105190001092B9031092BB031092BA0300EE10E014
:1051A000F80180818B7F808388818160888342E0E1
:1051B00060E080E00E941428E1EEF0E080818E7FC4
:1051C0008083E2EEF0E0808181608083808188606E
:1051D0008083F80180818E7F8083888180618883CD
:1051E000DF91CF911F910F910895E8EDF0E080815C
:1051F0008F7E8083E7EDF0E080818160808384E0B2
:1052000082BF81E08093BC030E94B2280895E8ED3C
:10521000F0E080818E7F80831092E20008951092EA
:10522000DA001092E10008951F920F920FB60F92CC
:1052300011242F933F934F935F936F937F938F939B
:105240009F93AF93BF93EF93FF938091E10082FF11
:105250000BC08091E20082FF07C08091E1008B7F4C
:105260008093E1000E94732B8091DA0080FF19C0C7
:105270008091D80080FF15C08091DA008E7F8093E6
:10528000DA008091D90080FF96C080E189BD82E17B
:1052900089BD09B400FEFDCF81E08093BD030E946B
:1052A000D1248091E10080FF19C08091E20080FF4D
:1052B00015C08091E2008E7F8093E2008091E20031
:1052C00080618093E2008091D80080628093D80052
:1052D00019BC85E08093BD030E94E5248091E10024
:1052E00084FF2BC08091E20084FF27C080E189BD4C
:1052F00082E189BD89B5982F917080FFFBCF8091A5
:10530000D8008F7D8093D8008091E1008F7E8093BC
:10531000E1008091E2008F7E8093E2008091E200C4
:1053200081608093E2008091B903882309F449C029
:1053300084E08093BD030E94EE248091E10083FF0E
:1053400029C08091E20083FF25C08091E100877F22
:105350008093E10082E08093BD031092B9038091B5
:10536000E1008E7F8093E1008091E2008E7F809348
:10537000E2008091E20080618093E20042E060E020
:1053800080E00E9414288091F00088608093F000F3
:105390000E94E224FF91EF91BF91AF919F918F9175
:1053A0007F916F915F914F913F912F910F900FBE21
:1053B0000F901F90189519BC1092BD030E94DF2416
:1053C00070CF8091E30087FD93E09093BD03B3CF4E
:1053D0001F920F920FB60F9211242F933F934F936A
:1053E0005F936F937F938F939F93AF93BF93CF936D
:1053F000DF93EF93FF93D091E900DF708091EC0091
:10540000C82FC17080FDC0E81092E9008091F000C3
:10541000877F8093F00078940E942C2A1092E900F4
:105420008091F00088608093F000CD2BCF70C09306
:10543000E900FF91EF91DF91CF91BF91AF919F91E3
:105440008F917F916F915F914F913F912F910F902D
:105450000FBE0F901F901895AAE2B0E0E2E3FAE2C7
:105460000C94402C8EEB93E02091F100FC012193F1
:10547000CF01F3E0863C9F07B9F70E941825809181
:10548000E80083FF1EC18091BE039091BF039A3054
:1054900008F017C1E92FF0E0EB55F24D0C94F32B17
:1054A000803899F0823809F00CC18091C2038F7066
:1054B000873008F006C18093E9008091EB0085FBFE
:1054C000882780F91092E90006C08091BA03909174
:1054D000BB03911182609091E800977F9093E80060
:1054E0008093F1001092F1008091E8008E77E5C082
:1054F000882309F4D3C0823009F0E3C08091C0034F
:105500008111D6C08091C2038F702FEF280F2630F3
:1055100008F0D7C08093E9002091EB0020FFC8C0BD
:10552000933031F48091EB0080628093EB00C0C037
:105530009091EB0090619093EB0021E030E001C08E
:10554000220F8A95EAF72093EA001092EA008091F0
:10555000EB008860EACF8111B4C01091C0031F77BF
:105560008091E3008078812B8093E3008091E800B4
:10557000877F8093E8000E9448288091E80080FFA0
:10558000FCCF8091E30080688093E30082E01111FA
:1055900083E08093BD0395C08058823008F091C0AD
:1055A0008091C0039091C1038C3D23E09207A1F547
:1055B00083E08A838AE289834FB7F894DE011396E9
:1055C00020E03EE051E2E32FF0E050935700E491F9
:1055D00020FF03C0E295EF703F5FEF708E2F90E0E9
:1055E000EA30C0F0C7968D939D932F5F243159F711
:1055F0004FBF8091E800877F8093E8006AE270E007
:10560000CE0101960E9457278091E8008B77809306
:10561000E80057C0C096E7CF6091C2037091C30302
:10562000AE014F5F5F4F0E944926BC01892B09F4F0
:1056300048C09091E800977F9093E80089819A8113
:105640000E94B527E1CF8038E1F58091E800877F9F
:105650008093E8008091B9038093F10045CF8111D8
:1056600030C09091C003923060F58091E800877F50
:105670008093E8009093B9030E9448288091B90371
:10568000882311F084E005C08091E30087FDFACF04
:1056900081E08093BD030E94F92413C08091C00370
:1056A000813079F481E0933009F080E08093BB038E
:1056B0001092E9008091E800877F8093E8000E94C3
:1056C00048288091E80083FF0AC08091E800877F26
:1056D0008093E8008091EB0080628093EB00AA96B3
:1056E000E3E00C945C2C0895CF938091BD03882354
:1056F000A1F0C091E900CF709091EC00892F8170EA
:1057000090FD80E8C82B1092E9008091E80083FDAD
:105710000E942C2ACF70C093E900CF910895991B65
:1057200079E004C0991F961708F0961B881F7A9598
:10573000C9F78095089587FB082E062687FD819579
:1057400067FD61950E948F2B0EF4919507FC819562
:105750000895AA1BBB1B51E107C0AA1FBB1FA617B8
:10576000B70710F0A61BB70B881F991F5A95A9F70A
:1057700080959095BC01CD01089597FB072E16F4F6
:10578000009407D077FD09D00E94A92B07FC05D013
:105790003EF4909581959F4F0895709561957F4F48
:1057A0000895A1E21A2EAA1BBB1BFD010DC0AA1F62
:1057B000BB1FEE1FFF1FA217B307E407F50720F07A
:1057C000A21BB30BE40BF50B661F771F881F991FF5
:1057D0001A9469F760957095809590959B01AC013E
:1057E000BD01CF010895EE0FFF1F0590F491E02D4C
:1057F00009946927962769277827872778270895A6
:105800000E94082C332312F48A1B9B0B0C94192C36
:10581000A29FB001B39FC001A39F700D811D1124F1
:10582000911DB29F700D811D1124911D08950E943C
:10583000082CB7FF0895821B930B08950E94082C33
:10584000A59F900DB49F900DA49F800D911D1124D4
:105850000895B7FF0C941E2C0E941E2C821B930BE4
:1058600008952F923F924F925F926F927F928F9204
:105870009F92AF92BF92CF92DF92EF92FF920F93DF
:105880001F93CF93DF93CDB7DEB7CA1BDB0B0FB6E9
:10589000F894DEBF0FBECDBF09942A8839884888A6
:1058A0005F846E847D848C849B84AA84B984C8843C
:1058B000DF80EE80FD800C811B81AA81B981CE0F33
:1058C000D11D0FB6F894DEBF0FBECDBFED01089518
:1058D0008F929F92AF92BF92CF92DF92EF92FF9200
:1058E000CF93DF93EC01688179818A819B81611577
:1058F00071058105910521F464E279ED8BE597E06E
:105900002DE133EF41E050E00E94262D49015A017C
:105910009B01AC01A7EAB1E40E941E2C6B017C0143
:10592000ACEEB4EFA50194010E942C2CDC01CB015C
:105930008C0D9D1DAE1DBF1DB7FF03C00197A109B2
:10594000B04888839983AA83BB839F77DF91CF91E7
:10595000FF90EF90DF90CF90BF90AF909F908F908F
:1059600008950E94682C089580E091E00E94682CC0
:105970000895B0E0A0E08093000190930101A0930E
:105980000201B09303010895FC014150504030F0F2
:1059900001900616D1F73197CF01089588279927EE
:1059A0000895FB01DC0104C08D910190801921F460
:1059B00041505040C8F7881B990B0895F999FECFC4
:1059C00092BD81BDF89A992780B50895A6E1B0E00F
:1059D00044E050E00C94182DA8E1B0E042E050E023
:1059E0000C94182D262FF999FECF92BD81BDF89AFF
:1059F000019700B4021639F01FBA20BD0FB6F89413
:105A0000FA9AF99A0FBE08950396272F0E94F32C55
:105A10000E94F22C252F0E94F32C242F0C94F32C9F
:105A20000196272F0E94F32C0C94F22CDC01CB0161
:105A3000FC01F999FECF06C0F2BDE1BDF89A31969E
:105A400000B40D9241505040B8F70895052E97FBD1
:105A50001EF400940E943D2D57FD07D00E94D12BCB
:105A600007FC03D04EF40C943D2D50954095309595
:105A700021953F4F4F4F5F4F0895909580957095BA
:105A800061957F4F8F4F9F4F0895F894FFCFA307E5
:105A9000A307D407D40761080308030803087D0897
:105AA000E408F308F308FD1C091D301D3C1D471DCB
:105AB000521D551D581D5B1DA41DA41D5E1D621D9C
:105AC0006A1D771D841D871D8A1D971DFB1EF21EF2
:105AD000FE1EF01E4B1F4B1FF01E4B1F4B1F1A1FAD
:105AE0004B1F251F301F4B1F4B1F4B1F4B1FF01E03
:105AF0004B1F4B1FF01E4B1F0C1F4B1F4B1F491FF3
:105B0000491F491F491F491F491F491F491F491F55
:105B10003B1F4B1FFB1EEE1E4B1F4B1F4B1F4B1FF4
:105B20004B1F4B1F4B1F4B1F4B1F4B1F3B1F4B1F35
:105B30004B1FF01E4B1F411F411F411F411F411FA3
:105B4000411F411F411F411F3B1F502A782A612BD3
:0E5B5000782A612BAB2ACC2A612B232B2F2B1A
:105B5E00010000005C020101020018001818011972
:105B6E001A1B1C1D1E1F2021222E243224A624A106
:105B7E00249C24312401E200E900EA00B500B600BD
:105B8E00B700CD008301CC008A019201940121025D
:105B9E00230224022502260227022A02B300B400A1
:105BAE006F007000818283E200E900EA00B500B662
:105BBE0000B700CD008301CC008A0192019401212F
:105BCE0002230224022502260227022A02B300B46F
:105BDE00006F007000818283C6309291909336F1EF
:105BEE00F4F5F6F7676635349496979531F0000123
:105BFE00020202020606060909090909090F0F0F1A
:105C0E000F0F0F1515151819191919191919191921
:105C1E0019232425252525252540226DA80719079A
:085C2E003B07BE06D706F7068E
:00000001FF
